:0E000000BBC0FECFFDCFFCCFFBCFFACFF9CFB8
:10000E00F8CFF7CFF6CFF5CFF4CFF3CFF2CFF1CFC6
:10001E00F0CFEFCFEECFEDCFECCFEBCFADC1E9CF41
:10002E00E8CFE7CFE6CF1027E80364000A0001000F
:10003E000010000110000100C409881384030D484C
:10004E00565F436F6E7665727465723A2025640052
:10005E000D565F544F5F50574D202A2031305E337E
:10006E00203D202564000D4144435F544F5F5620D0
:10007E002A2031305E33203D2025640D000D45527F
:10008E00523A20496E636F727265637420636F6DAE
:10009E006D616E640D000D4552523A20496E636FCC
:1000AE00727265637420616464726573730D004DC2
:1000BE00656173757265204D494E20766F6C746163
:1000CE00676520000D4552523A20496E636F727279
:1000DE0065637420766F6C746167650D004D6561A4
:1000EE0073757265204D415820766F6C746167652B
:1000FE0020004D656173757265204D454449554D1F
:10010E0020766F6C746167652000414443203D206A
:10011E002564000D4144435F544F5F56202A203121
:10012E00305E33203D2025640041444452203D2062
:10013E0025640D0048563D25640D004856204F4657
:10014E00460D004856204F4E0D004F43523142206F
:10015E003D2025640D0001002D4E414E00494E46B6
:10016E00000001008C0164010000F894EE27EFBB43
:10017E00E5BFF8E1A895A4B7A77FA4BFF0936000F0
:10018E00E09360008DE0A2E0BB27ED938A95E9F73E
:10019E0080E092E0A0E0B1E0ED930197E9F7E0E7AF
:1001AE00F1E085919591009761F0A591B59105903B
:1001BE001590BF01F00105900D920197E1F7FB013B
:1001CE00F0CFE0E0EEBBEFEFEDBFE2E0EEBFC0E858
:1001DE00D1E066C1AA935B9AE881E093C6008DD305
:1001EE00E074E9F38AD3E064E093C0005B980AC040
:1001FE00AA93A881AD3021F4ADE0ECDFAAE0EADFEE
:10020E00A881E8DF21960895DED500E010E07BD2CC
:10021E004E2EA42D61D3E03069F0A895AAE0A09FE0
:10022E00F001A19FF00D8F01E42D6AD3F0970E0F10
:10023E001F1F01C001C0EBCFF801CFD50895E0E03C
:10024E00E5B9E4E0E4B9E0E0E8B9E7B9E0E2EBB93A
:10025E00EAE2EAB9E0E0E4BDE5BDE6BDE7BDE8BD32
:10026E00E3E3E0938000E9E1E0938100E0E0E093D6
:10027E008500E0938400E0938700E0938600E9E038
:10028E00E0938900E4ECE0938800E0E0E0938B00DB
:10029E00E0938A00E093B600E093B000E093B100E3
:1002AE00E093B200E093B300E093B400E0936900F2
:1002BE00EDBBE0936800E0936E00E0936F00E09377
:1002CE007000E093C000E8E1E093C100E6E0E09347
:1002DE00C200E0E0E093C500EDE4E093C400E0E886
:1002EE00E0BFE0E0E0937B00E0937F00E2E0E0938C
:1002FE007E00EFE8E0937A00E1ECE0937C00E0E032
:10030E00ECBDE093BC00A895E8E3E0936000E8E262
:10031E00E09360000895F6D2E981E0938B00E881C6
:10032E00E0938A0022960895EDD24DD5A5E0B0E077
:10033E0017D5AA81BB8109D5EA1BFB0BE6D27F93A9
:10034E006F93FF93EF93E5D2AF91BF918F919F91F2
:10035E0013D4ABD38F01D801DEDFF894DED27894BC
:10036E0039D524960895F894D8D27894E0918A01DC
:10037E00E030E1F3EAD208950A921A92FA926A9361
:10038E007A938A939A93AA93BA93EA93FA93EFB7CE
:10039E00EA9315D5E0917800F0917900AF01FA015A
:1003AE00D9D2E1D280D4E0938401F0938501609399
:1003BE00860170938701A0E8B1E0B4D4EF5FFF4FE0
:1003CE006F4F7F4FB4D4E13DA2E0FA07A0E06A0779
:1003DE00A0E07A0708F453C0BDD2E1EDF2E060E090
:1003EE0070E077D4E0938801F0938901E0E0E09328
:1003FE008401E0938501E0938601E0938701E09309
:10040E008001E0938101E0938201E0938301E1E0BA
:10041E00E0938A01E0918B01E03089F596D275D296
:10042E007F936F93FF93EF93A1D2AF91BF918F9173
:10043E009F91A0D28F01E0918B00FE2FE0E0DF01B3
:10044E00E0918A005DD2EA0FFB1F9F0196D20E1734
:10045E001F0720F4243CE9E03E0708F003C02F5F9D
:10046E003F4F0BC08AD2E017F10720F4002402168A
:10047E00030608F002C021503040D9014CDF81D272
:10048E00A5D42696E991EFBFF991E991B991A99179
:10049E009991899179916991F9901990099018958E
:1004AE002697CDDEA0EDB7E0C9D2ECE4F0E06FD236
:1004BE0071D2FF276627772771D275D278D27CD278
:1004CE00E4E7F0E064D252D272D276D256D2DF0195
:1004DE002BDF5D9A789455D2A8950FD2E07809F467
:1004EE0010C111D1AE2F01D21E2F133461F0113471
:1004FE0051F0163541F0183431F0133521F0173420
:10050E0011F0103509F404C0EBE8F0E058D2E4CF56
:10051E005BD240D2D901F4D1EA17FB0729F0EDEFF7
:10052E00F0E0E217F30709F404C0E4EAF0E047D282
:10053E00D3CFE12FE5D1E334A0E0FA0709F081C073
:10054E00E1E045D2A0E0B0E0E6DEEDEBF0E037D240
:10055E00A8955ADEAF01042E052A21F04938E3E1B1
:10056E005E0718F037D239D2B7CFA4ECB9E0D3DE9C
:10057E00EBEEF0E024D2A89547DEEC83FD832FD27C
:10058E00309731F0AC81BD81A838E3E1BE0718F099
:10059E0021D223D2A1CFA2EEB4E0BDDEE0E0F1E0A5
:1005AE000ED2A89531DEEA83FB83309759F0AA81EB
:1005BE00BB81A417B50730F012D2AA81BB81EA170E
:1005CE00FB0718F407D209D287CFA895CCDEE883B3
:1005DE00F983E8E1F1E0DBD1EA81FB81C4D1DED120
:1005EE00FA01A5E0B0E0D3D3FAD1A3E0B0E0CFD3C7
:1005FE00F6D1E41BF50B89D1A0E0B0E48CE195E4D3
:10060E0009D3A7E0B0E0BBD3CED1D1D1D5D1EA8109
:10061E00FB817BD1DF01CB01E881F98176D1FAD262
:10062E00ABE0B0E0ACD3E1E2F1E0B1D19FD1BFD10C
:10063E00C3D1D3D1A2D1DF0177DEE9E8F0E0BFD19B
:10064E0060C0E134A0E0FA07C1F4E0E2E41569F419
:10065E00BBD1022E032A21F02D3FE0E03E0708F029
:10066E0004C0E22FA0E0B0E09AD3E7E3F1E08FD12F
:10067E0091D1FF276627772740C0E635A0E0FA071D
:10068E00A9F4A2D12938E3E13E0710F028E833E1BE
:10069E002438E3E03E0710F424E833E0F901A1E04A
:1006AE00B0E075D3D90140DE9DD125C0E834A0E07D
:1006BE00FA0711F497D11FC0E335A0E0FA0729F429
:1006CE005D98E9E4F1E07BD11CC0E734A0E0FA07C5
:1006DE0029F45D9AE1E5F1E072D113C0E035A0E0B6
:1006EE00FA0779F4E1E073D16FD1D90114DEE8E5B0
:1006FE00F1E04DD1F9016627772722D384E0CED0E1
:10070E002696EACEFFCFF9D0E078E9F3E091C60065
:10071E000895F8D0AA816CDDA881B981ED91FD9183
:10072E003196FE93EE9323960895ECD0249747D3FB
:10073E0010E0AA85BB85E0E0F0E0ED93FC93E8893C
:10074E00F9893196E88BF98B51D109F4A1C0E12FCB
:10075E00E03031F4353211F411E001C04CD197C0C4
:10076E00E13081F4353211F446D190C012E020E030
:10077E0000E03B3211F42BE28AC0303211F420E259
:10078E0086C002C0E23031F4303319F4006115E056
:10079E007EC003C0E53009F07AC0E32FE33639F4AA
:1007AE0031D133D12FD1A481AA9333D16FC0E33786
:1007BE0069F435D136D1AE81BF81ED91AE83BF8361
:1007CE003E2FE03011F017D1F6CF60C0E03761F464
:1007DE0026D127D1EE81FF813196EE83FF8306D19C
:1007EE0011F009D1F7CF52C0E43611F0E93611F409
:1007FE00016002C0E53719F4E4E3F0E009C0E83522
:10080E0011F4026003C0E83709F040C0EEE3F0E0F7
:10081E00EE83FF8300FF0DC002D10AD1552322F4CF
:10082E00FA0146D2AF012DE2203011F02A93F1D019
:10083E0002C0F5D0FDD030E3EE81FF817DD2E88796
:10084E00F987EE81FF813296EE83FF83E885F98585
:10085E004E175F0730F03F5FA885B9854A1B5B0BCB
:10086E00F5CF04FD06C0313320F4A885B985119764
:10087E0049F400613A3328F001FF02C0395F01C02C
:10088E00395DB9D0A885B9851297A8F610E057CF73
:10089E00AA85BB8543D29AD262960895FF92F82E0E
:1008AE00269791D2DE011496FAD18D01E0E0EC8309
:1008BE00ED83EE83EF83DE011896F1D12FD267D050
:1008CE001A930A93E0E9F3E062D0DE0118962DDF69
:1008DE0081D22896FF900895AA93E1E0F991F03322
:1008EE0010F0FA3308F0EE270895AA93E991E13655
:1008FE0018F0EB3708F4E0520895E091C000089527
:10090E00F0E00895BA93AA9308956627772706D143
:10091E000895A7E0B0E020D20895E0E0E0938401CE
:10092E00E0938501E0938601E0938701E0938001D7
:10093E00E0938101E0938201E0938301E0938801CB
:10094E00E0938901E0938A010895E0918801F09186
:10095E0089010895A0918401B0918501809186014D
:10096E00909187010895662777270895ABE0B0E050
:10097E00F3D1089501D199D00895A1E0B0E0F0D15E
:10098E000895E0917A00E064E0937A000895FA9376
:10099E00EA930895A0E0B0E0E7D10895D1D184E0C4
:1009AE007DDF26960895EEE5F0E0F1DFB2CFA0E010
:1009BE00B0E08AE794E4DECFD6DFD5DFEFCFE7DF16
:1009CE0080E06CDF229608951FDC9F010895E0936E
:1009DE008B010895E2EDF0E0F2CFE0E0F8CFEC818C
:1009EE00FD810895E2E4F1E0D2DFC7CF3197E491C3
:1009FE003E2FE03008953A93AB85BC85ED85FE859C
:100A0E0009950895EE85FF8508953497EE87FF8743
:100A1E000895AB85BC85ED85FE8509950895F2DFB9
:100A2E00F4CFAE85BF85149679D1EE83FF830895FA
:100A3E00AE85BF8514964D915C910895109639F050
:100A4E0088EB9BE00197F1F7A8951197C9F70895E8
:100A5E00552342F4503811F4E0FF04C03196691F5B
:100A6E00791F6BF050E8572711F45F9373C05F3F07
:100A7E0031F0660F000C57956795752F08955F93AB
:100A8E0000200AF073C06CC050E8192E1522880F92
:100A9E00991F9527550F879550E8072E0522660F4B
:100AAE00771F7527550F67950895689401C0E894D0
:100ABE005F93F2DF703818F07F3F08F44BC056E1B9
:100ACE00571BAAF4519558300EF4593030F0EFEF11
:100ADE00FFEF6FEF7FE777F91AC077275523B9F04D
:100AEE00EE0FFF1F661F771F5A95D1F710C077279D
:100AFE00583028F0EF2FF62F672F5850F9CF552387
:100B0E0031F076956795F795E7955A95D1F70020D0
:100B1E000AF4D2D05F910895689401C0E89430979A
:100B2E0060407040B1F0002426F0772312F4009458
:100B3E00C3D0172E7EE1112032F07A95EE0FFF1FF3
:100B4E00661F111CF9CFEF2FF62F612D5F938ADFF1
:100B5E005F910895EE27FF27662777275F91089507
:100B6E00EFEFFFEF6FE77FEF5F910895EFEFFFEF8E
:100B7E006FE77FE75F9108955F9386DF703851F3DB
:100B8E00903841F301240894791F23F41CF30020BC
:100B9E003AF3ECCF0F921F932F933F934F9311275E
:100BAE0022279927689FA0018F9F302D410D591F35
:100BBE006B9F300D411D591F8E9F27D0BF9F25D093
:100BCE006A9F23D0BE9F1DD0AF9F1BD0AE9F110D2D
:100BDE00291F391F491F591FE32FF42F652F522F3D
:100BEE004F913F912F911F910F9066232AF0550F31
:100BFE00EE1FFF1F661F02C073954BF229DF5F9138
:100C0E000895100D211D391F02C0200D311D491FE1
:100C1E00591F08955F9338DF703821F411200AF4BC
:100C2E009FCFA4CF903809F495CF01240894970B49
:100C3E001BF4D4F30020F3CF792F1F932F933F9300
:100C4E004F9311241127222733274427552790E24B
:100C5E00AE17BF078607410730F0AE1BBF0B860BE2
:100C6E00410B089401C08894551F221F331F111C7D
:100C7E00AA1FBB1F881F441F9A9551F7F901612DBA
:100C8E004F913F912F911F91662332F0550FEE1F1A
:100C9E00FF1F661F7A9543F2DBDE5F9108950024F5
:100CAE00AF0DB01D0895EA0FFB1F681F791F089541
:100CBE00F195E195F0400895F09560957095E19568
:100CCE00FF4F6F4F7F4F08956F2F660F660B762F76
:100CDE0008953F934F935F93002411244427552783
:100CEE0030E2AA0FBB1F881F991F001C111C441F46
:100CFE00551F0E1A1F0A460B570B28F40E0E1F1EF9
:100D0E00461F571F01C0A1603A9559F7FD01BC015E
:100D1E00D001CA015F914F913F910895ED91FC91E1
:100D2E0011970895ED91FD916D917D9108957E93AA
:100D3E006E93FE93EE9308950590F491E02D089531
:100D4E007A936A93FA93EA9308951B2EBF2FF12D8F
:100D5E001A2EAE2FE12D0895129602D0BF011297D2
:100D6E00119602D0FE2F1197F999FECFFF93FFB780
:100D7E00F894A1BDF89AE0B5FFBFFF91089507D092
:100D8E0012960F01FB0103D0F0011297089507D0C0
:100D9E001196EF93EF2F03D0EF9111970895F99BD2
:100DAE0002C0A895FCCF9FB7F894A1BDF89A80B564
:100DBE00E81719F0E0BDFA9AF99A9FBF08955A9371
:100DCE004A933A932A931A930A9308955D814C811C
:100DDE003B812A81198108810895099119910895FD
:00000001FF
